:1001AF008F22ED2400B40800504FFC232C9001C087
:1001BF00730201DA0201E00201E60201EC0201F230
:0B01CF000201F80201FE020204802E73
:1001DA00A22392108028A22392118022A223921293
:1001EA00801CA22392138016A22392148010A223A9
:1001FA009215800AA22392168004A2239217AF2294
:01020A0022D1
:10020B008F22C221ED2400B40800504FFC232C9008
:10021B00021E7302023802023E02024402024A022A
:0D022B00025002025602025C020262802EA6
:10023800A21092218028A21192218022A21292213A
:10024800801CA21392218016A21492218010A2155C
:100258009221800AA21692218004A2179221A2213B
:010268002273
:10026900C283C282A22492818F21120F95858017A1
:1002790053170F752200A20F9214A20E9215A20D08
:100289009216A20C9217E5224517F51785178012C9
:100299000F95D283120F95202414E5216401600B78
:1002A900E52164026005E521B40303120F82C283CC
:1002B900202414E5216401600BE52164026005E551
:1002C90021B40303120F82120F95E517540FF51786
:1002D900752200A20B9214A20A9215A2099216A2E3
:1002E900089217E5224517F517851780120F95D241
:1002F90083120F95202414E5216401600BE5216424
:10030900026005E521B40303120F82C2832024147D
:10031900E5216401600BE52164026005E521B40370
:0B03290003120F82120F95120F952295
:100334007F01120F53C283C282C281752128858036
:100344002575260FE5265525F525752200A20F9261
:1003540014A20E9215A20D9216A20C9217E5224534
:1003640025F525852580120F82D283120F82C28340
:10037400120F827580F0120F82120F82C2247F281E
:10038400120269C2247F28120269C2247F01120268
:1003940069C2247F03120269C2247F06120269C261
:0E03A400247F0C120269C2247F171202692204
:0E03B200E52A700122750800E508640A607DE6
:0903C000750900E50964056044BB
:1003C900D2B2750A0175F005E509A42464FBE43588
:0C03D900F0F5F0E4B5F005E50A6B6004F7
:1003E500050A80E5C2B2750A0175F005E509A42480
:1003F50064FBE435F0F5F0E4B5F005E50A6B60045F
:10040500050A80E5050980B6750900E509640560FA
:0104150022C4
:0B041600D2B2750A01E50A64646004BC
:0F042100050A80F6D2B2750A01E50A6464600428
:0E043000050A80F6050980D805080203BA22E5
:0B043E00E52A7001227E00BE50012262
:09044900D2B27F01BFC80280039A
:0C0452000F80F8C2B27F01BFC802800317
:06045E000F80F80E80E1A2
:0B046400E52A7001227E00BE5A012232
:09046F00D2B27F01BFB402800388
:0C0478000F80F8C2B27F01BFB402800305
:060484000F80F80E80E17C
:0B048A00E52A7001227E00BE64012202
:09049500D2B27F01BF9602800380
:0C049E000F80F8C2B27F01BF96028003FD
:0604AA000F80F80E80E156
:0A05FC008F44E4F54512141F50036C
:0806060012143112141F5011EF
:10060E007B057A0479B0120F9F7F0A120F53E4FF15
:0D061E002212144EC2227FA0121517501197
:10062B007B057A0479D1120F9F7F0A120F53E4FFD7
:10063B0022AF4412149812144ED2227FA012151717
:02064B0050114C
:10064D007B057A0479F2120F9F7F0A120F53E4FF94
:0F065D00221214E28F45121488121463AF452243
:09066C008F448D4512141F500348
:0806750012143112141F500F82
:10067D007B057A057913120F9F7F0A120F532212F1
:0B068D00144EC2227FA0121517500F60
:100698007B057A0479D1120F9F7F0A120F5322AF7C
:0606A80044121498500FEB
:1006AE007B057A057934120F9F7F0A120F5322AF02
:0606BE0045121498500FD4
:1006C4007B057A057955120F9F7F0A120F53221268
:0606D4001463120F8222E4
:1006DA00E4FEFD8F04BF6301D340037F6322EC7005
:0706EA0003E4FF22EC600AAB
:0506F1001C0EBE0AF81A
:0F06F600E4FE0D80F3ED75F010A4FDEE4DFF2234
:100705008F448C458D46754701E4FCF54875494A8B
:10071500754C01F54D754E4FAE45AF467D641200E3
:1007250044EEAB4CAA4DA94E12014BEF1200D9195C
:10073500B9FF011A12014FFE120120FFE4FC7D648E
:10074500120008E546C39FFFE5459EAB47AA48A9A9
:100755004912014BEF1200D9A22292237512017999
:1007650050E4FA7B01AD44120FFCA22292237512CC
:0F07750002794BE4FA7B01E54404FD120FFC22EC
:100784008F448C458D46754701E4FCF54875494A0C
:10079400754C01F54D754E4FAE45AF467D64120064
:1007A40044EEAB4CAA4DA94E12014BEF1200D919DD
:1007B400B9FF011A12014FFE120120FFE4FC7D640F
:1007C400120008E546C39FFFE5459EAB47AA48A92A
:1007D4004912014BEF1200D9A22292237512027919
:1007E40050E4FA7B01AD44120FFCA222922375124D
:1007F40002794BE4FA7B01E5442402FD120FFC224A
:10080400E404FB14FA7912EE12014BEF1200D9C280
:10081400A0D2A3D2A4C2A1851222A21392A2D2A1D1
:10082400C2A1A21292A2D2A1C2A1A21192A2D2A149
:10083400C2A1A21092A2D2A1C2A1851322A2179290
:10084400A2D2A1C2A1A21692A2D2A1C2A1A2159221
:10085400A2D2A1C2A1A21492A2D2A1C2A1A2139215
:10086400A2D2A1C2A1A21292A2D2A1C2A1A2119209
:10087400A2D2A1C2A1A21092A2D2A1C2A1C2A37F5C
:0508840001BF2001226C
:030889000F80F9E4
:0F088C00E4FDA2B382B482B55002C22020201E28
:03089B0020B30780
:0A089E007D02D22012043E20B407B0
:0A08A8007D01D22012048A20B5075A
:0A08B2007D03D2201204648D07229A
:1008BC00754010E4F541754210F543F544F545E5F6
:0808CC0044B41004E545603757
:0A08D400AE44AF4512080420B61030
:1008DE00E542B4100BE543B400068544428545431A
:0308EE0020B71020
:1008F100E540B4100BE541B400068544408545410F
:0B0901000545E54570C4054480C02298
:10090C008F4D8B4E8A4F89508D518C528853755414
:10091C0001755506E4F556F557120F9FE555B406CB
:06092C000280030209E451
:0A09320012088C8F58E558B4017DBF
:10093C00E4F556F5570554E54D2401FBE43400F578
:10094C00F0E4B5F008E554B50303E4F554E554B40C
:10095C000302803A500CE554601314601B1460239E
:0D096C00804BE55424FC603114603980405C
:100979007B057A10798F120F9F8035AB4EAA4FA94C
:1009890050120F9F802AAB51AA52A953120F9F8070
:100999001FAB44AA45A946120F9F8014AB47AA482A
:1009A900A949120F9F8009AB4AAA4BA94C120F9F64
:1009B900E558B40203855455E558B40303E4F555E5
:1009C900AA56AB570557E55770020556BA0706BB35
:0E09D900D003E4F555120F82020928AF552213
:1009E7008E048F05E4FE7F0A1200088E448F45AE01
:1009F70044AF45AD2C7C00120044EF252BF545E4B0
:080A07003EF544AE44AF452268
:0F0A0F007B057A1379B1120F9F7F1E120F5322AE
:100A1E007544057545057546767547057548057522
:100A2E004976754A05754B05754C767F027B057ABE
:100A3E001379517D057C13787112090C8F0DE50D1C
:080A4E00146005146007800824
:100A5600E4F52A8003752A017F02AD2A12066C226C
:100A66007B057A12792F120F9FC290E4F50DE50DE2
:040A76006402602D89
:100A7A0012088C8F0DE50DB4030122E50DB401EACD
:030A8A0020900DAC
:0D0A8D00D2907B057A12794F120F9F80DA0C
:100A9A00C2907B057A12792F120F9F80CDE50DB493
:100AAA000301221208BC85420E85430F7B057A1288
:100ABA00796F120F9FC2227F05AC0EAD0F12078409
:100ACA007F0A120F537B057A12798F120F9FC290F9
:090ADA00E4F50DE50D6402602D48
:100AE30012088C8F0DE50DB4030122E50DB401EA64
:030AF30020900D43
:0D0AF600D2907B057A1279AF120F9F80DA43
:100B0300C2907B057A12798F120F9F80CDE50DB4C9
:100B13000301221208BC8542108543117B057A121A
:100B230079CF120F9FC2227F05AC10AD111207843B
:100B33007F0A120F53E511C3950FFFE510950EFEC3
:100B4300E4FC7D0A1200448F2CAC0EAD0FE4FE7F53
:100B53000A120008AD2C7C0012004474C8C39FF530
:100B63000FE49EF50E850F2B7B057A1279EF120F9A
:100B73009FC223751203792CE4FA7B017D07120FC0
:100B8300FCD223751203792BE4FA7B017D0B120F40
:100B9300FC7F64120F53E52924FFC3332403FFAD05
:100BA3002C12066CE52924FFC3332404FFAD2B125A
:030BB300066C22AB
:100BB6007544057545117546CF7547057548117518
:100BC60049EF754A05754B05754C767F047B057AAA
:100BD60011798F7D057C1178AF12090C8F0DE50D0B
:0E0BE60014600B14600D14600F146011801267
:100BF400752901800D752902800875290380037504
:100C040029047F01AD2912066CE52924FFC333248E
:100C140003FF1205FC8F2CE52924FFC3332404FFB2
:060C24001205FC8F2B22DB
:100C2A007B057A1379F3120F9FE4F50DE50D640342
:020C3A006064F4
:100C3C001208BCC2227F04AC42AD43120784C2220C
:100C4C007F0BAC40AD41120784D223751203792C73
:100C5C00E4FA7B017D03120FFCD223751203792B6E
:100C6C00E4FA7B017D08120FFCAE42AF431209E798
:100C7C008E428F43D2227F0EAC42AD431207051237
:090C8C00088C8F0DE50DB401A1E7
:030C9500209004A8
:040C9800D290809ADC
:050C9C00C290809622C9
:070CA100E4F50BE50B706C9C
:100CA80075440575451375463175470575481375BF
:100CB8004991754A05754B13754CD27F057B057AAA
:100CC80011796F7D057C12780F12090C8F0CE50CD9
:100CD800B403028028500CE50C60131460151460EE
:0E0CE800178027E50C24FC601914601B80AEF9
:100CF600750B0180A9120BB680A4120A66809F129A
:0F0D06000A1E809A120A0F8095120C2A809022E2
:100D1500E4FFFD12066CE4F508E5086401700302C2
:020D25000DF5CA
:100D27001208BCAE42AF431209E78E428F43AC4074
:100D3700AD41E4FE7F0A1200088E408F41AE40AFFE
:100D470041E4FC7D9B120044EF248CF541E43EF521
:0C0D570040B54206E541B54301D3400D14
:0D0D63007B057A1079CF120F9FC290800B94
:100D70007B057A1079EF120F9FD290C2227F0DACC3
:100D800042AD43120705D2227F05AC40AD411207A8
:100D900005E542B40106E543B49001D340097B0563
:100DA0007A1079AF120F9F120F8212088CBF0102C6
:050DB0008003020D1E8E
:100DB500D2907544057545057546767547057548A0
:100DC50005754976754A05754B05754C767F027B29
:100DD500057A11790F7D057C11784F12090C8F0862
:100DE500E508B402028003020D1E120CA1020D1EBD
:0B0DF500E4FF7D0112066C120F822249
:100E0000D290E4FF7D0112066C7B057A11792F12D6
:080E10000F9F12088CEF7045E2
:100E18001208BCAE42AF431209E78E428F43E54247
:100E2800B40106E543B49001D34005E4F542F54327
:100E38007B057A11792F120F9FE542B40105E5432E
:050E4800B49000500B06
:100E4D00D2227F0DAC42AD43120705120F8280B541
:0A0E5D00E4FFFD12066C120F822262
:100E6700120F8275800F7590FF75A0FF75B0FFC2D6
:100E7700201203B21203347B057A057977120F9F8C
:0A0E870012088C8F25E525B4015AEE
:100E91007B057A057998120F9F7F0A120F53E4FFA1
:100EA100FD12066C7F017D0112066C7F027D01122D
:100EB100066C7F037D5E12066C7F047D2D12066C2D
:100EC1007F057D5912066C7F067D3212066C7F0705
:100ED1007D5612066C7F087D3712066C7F097D5E98
:100EE10012066C7F0A7D2D12066C7F011205FC8FA4
:100EF100297F021205FC8F2AE52924FFC33324032D
:100F0100FF1205FC8F2CE52924FFC3332404FF12B3
:100F110005FC8F2B7F05120F537B057A0579B912DA
:070F21000F9F7F05120F5323
:100F2800E4FF1205FC8F28E5286005146007800A95
:100F3800120D1580EB120E0080E67B057A0579DA32
:090F4800120F9FE4FFFD12066C7C
:020F510080FE20
:1004B000204552524F5220493243202020202020F4
:1004C00020202042555320425553592021202020DE
:1004D00000204552524F52204932432020202020F4
:1004E00020202020204E4F2041434B20212020203F
:1004F0002000204552524F522049324320202020D4
:1005000020202020206572726F7220726561642045
:10051000202000204552524F5220493243202020B3
:10052000202020202020425553204255535920217D
:1005300028772900204552524F522049324331201A
:10054000202020206572726F722077727974652086
:100550006279746500204552524F5220493243322D
:1005600020202020206572726F7220777279746566
:10057000206279746500002044455445435420525C
:1005800045534554202020202020205359535445C2
:100590004D202121212020002053455420544F205C
:1005A00020202020202020202020202044454641BB
:1005B000554C54202E2E2E20004449474954414C7E
:1005C000205354414E54494F4E20535452205645C7
:1005D0005253494F4E20332E31004572726F7220B4
:1005E0004D6F64652042797465212052657365748E
:0C05F0002073797374656D2120202000B9
:100F53007E01EF2401FBE43400F5F0E4B5F004EE88
:030F63006B601BA5
:070F6600751201E512601194
:090F6D00751301E513649B600497
:0C0F7600051380F6051280EB0E80D422DB
:060F82007F01BF320122D5
:0D0F88007E01BE320280030E80F80F80EF64
:060F95007F01BF320122C2
:040F9B000E0F80F8BD
:100F9F008B128A138914C2247F03120269751500FC
:100FAF00E5156410601BD224AB12AA13A914E51522
:100FBF00851582758300120159FF1202690515808C
:100FCF00DFC2247FC0120269751510E51564206019
:100FDF001BD224AB12AA13A914E5158515827583AC
:0D0FEF0000120159FF120269051580DF2272
:100FFC00E4F513F514F5158D16EBFDEAFCE9F81282
:0E100C0000F5FEEE1E60180513E513B40AF59C
:0A101A00E4F5130514E514B40AEB25
:10102400E4F514051580E430230CC224E51624BF2E
:10103400FF120269800AC224E516247FFF120269A6
:10104400E512B4030AD224E5152430FF120269E53F
:10105400126401600AD224E5142430FF120269D21A
:0A10640024E5132430FF1202692274
:10106E0020464C415348204E4F2020202020202047
:10107E0020202041434B4E4F574C4544474521209D
:10108E0000202020426570BD79BFC463C720202098
:10109E002020202020BD61B761E3202E2E2E20209F
:1010AE00204FC1B8B2BA6120E361BFC0B8BA6121A6
:1010BE0020A8504F424550A55462205041A4AD4542
:1010CE004D5465BCBE657061BF797061205858582B
:1010DE0043A963BF2E5858584320482E2042BABB0E
:1010EE002E5465BCBE657061BF797061205858582A
:1010FE0043A963BF2E5858584320482E42C3BABB4B
:10110E002EA963BF61BD6FB3B8BFC4207065B6B8FA
:10111E00BC202020204FA3A5E04148A5B1202020CF
:10112E00203E5065B6B8BC206FB6B8E361BDB8C7F7
:10113E003C5465BCBE657061BF79706120585858CB
:10114E0043202020A5B7BC65BD65BDB86520202015
:10115E0020202020BE617061BC65BF706FB320205F
:10116E002020A963BF61BD6FB3B8BFC420BFB8BE96
:10117E002020B661BB6120BE61C7BBC4BDB8BA61D9
:10118E002043BF61BDE36170BFBD6F6520B661BB1B
:10119E006F20BFB8BE203C534F4C4F4D4F4E3E209C
:1011AE002020204D65E3BD6F6520B661BB6F20200A
:1011BE002020E3BBB8BD612032302D333020BCBCC3
:1011CE002020204D65E3BD6F6520B661BB6F2020EA
:1011DE002020E3BBB8BD612031302D323020BCBCA5
:1011EE002043BE65E5B861BBC4BD6F6520B661BB6B
:1011FE006F2CBBB8B26F20E37079B46FB920BFB853
:10120E00BE20B063BFB8706FB3BA6120E565BEB8DB
:10121E00202020BF6570BC6FE361BFC0B8BA6120EB
:10122E0020A963BF61BD6FB3B8BF652032303020D7
:10123E00434861B47065B320424BA7B0AB4548211B
:10124E0020A963BF61BD6FB3B8BF652032303020B7
:10125E00434861B47065B32042AE4BA7B0AB45486E
:10126E00202020546FC0BA6120323030204320201D
:10127E002020B761E4B8BA63B8706FB361BD612165
:10128E0020A963BF61BD6FB3B8BF65203330302076
:10129E00434861B47065B320424BA7B0AB454821BB
:1012AE0020A963BF61BD6FB3B8BF65203330302056
:1012BE00434861B47065B32042AE4BA7B0AB45480E
:1012CE00202020546FC0BA612033303020432020BC
:1012DE002020B761E4B8BA63B8706FB361BD612105
:1012EE00202054616E67205858582020202020203E
:1012FE0020202020536D6573636820585858202095
:10130E0020003D3D3D3D3D3D3D3D3D3D3D3D3D3D59
:10131E003D3D3D3D3D3D3D3D3D3D3D3D3D3D3D3DEF
:10132E003D3D0020202020A4B379BA6FB36F652015
:10133E0020202020636FBE706FB36FB6E365BDB81B
:10134E0065202020202042C3BABBC6C0B8BFC4202F
:10135E002020202020202020B7B379BA2020202062
:10136E002020202020202020A4B379BA2020202065
:10137E002020202020202042BABBC6C065BD2020E0
:10138E002020202020A8706F63BC6FBF7065BFC483
:10139E002020202020A548AA4F50414D41E1A5B064
:1013AE0020202020205757572E5354522D42592E6D
:1013BE002020202020206E61726F642E72752020F6
:1013CE00202020002044454255472057494E444F87
:1013DE00572020202020205741524E494E47212190
:1013EE00212020200020563D5858585820523D5854
:1013FE00585858202054675858582D53585858202C
:06140E00543D585858003F
:061414007F01BFFA012276
:05141A00000E0F80F739
:05141F00D2A520A50884
:0D14240012141420A502D32230A501C3220A
:0514310012141F50170A
:09143600751201E512640A600E52
:0F143F00C2A6121414D2A6121414051280EC22A5
:10144E00D2A620A503121414D2A5C2A5121414C23A
:05145E00A61214142287
:10146300C2A630A503121414C2A5D2A6121414D214
:05147300A51214142273
:10147800C2A5121414D2A6121414C2A6121414224D
:10148800D2A5121414D2A6121414C2A6121414222D
:0B1498008F17751800E5186408602429
:1014A300AF177407C39518FD12020B5004D2A58021
:1014B30002C2A5121414D2A6121414C2A612141432
:1014C300051880D6D2A5121414D2A612141430A56E
:0F14D30004D2238002C223C2A6121414A2232221
:1014E200E4F512C2A6D2A5121414F513E51364088A
:0214F200602078
:1014F400D2A612141430A50FD223AF127407C395C9
:1015040013FD1201AF8F12C2A6121414051380DA50
:03151400AF1222F1
:101517008F1230220BD223AF12E4FD1201AF8F12CC
:06152700AF12121498221D
:030000000201A05A
:0F01A000758159E4787FF6D8FD75A0FF020E67D0
:1000D900CB30E11520E00FC083C08289828A83CBAF
:0C00E900F0D082D08322CBF322CBF72290
:1000F500ED30E11320E00EC083C08288828C83E05E
:10010500D082D08322E2226405700EC083C082882B
:0B011500828C8393D082D08322E622EC
:10012000EB30E11320E00EC083C08289828A83E035
:10013000D082D08322E3226405700EC083C08289FE
:0B014000828A8393D082D08322E722C2
:04014B0011D9215352
:04014F0031202153E7
:0601530009B900010A22B7
:10015900BB02030201884003BB040302017C400384
:0601690002016F02019487
:0D016F00E92582F582EA3583F583E49322C9
:0C017C008883E92582F8E6C8C583C82204
:0C018800E92582F582EA3583F583E02248
:0C0194008883E92582F8E2C8C583C822F0
:10000300E0A3FEE0FFEF8DF0A4CFC5F0CCA42CFC61
:09001300EE60038DF0A42CFE2226
:10001C00C2D1C2D5EE30E707D2D1D2D51200C9EC8D
:10002C0030E705B2D11200D112004430D1031200D6
:10003C00C930D5031200D122BC000EBE0032EF8DA8
:10004C00F08420D226FFADF0227B0075F008EF2F54
:10005C00FFEE33FEEB33FBEE9DEB9C4005FBEE9D80
:10006C00FE0FD5F0E9E4CECDCBCC227EFF7FFF2274
:10007C00EDB410005022EE8DF084FEEF54F045F0FC
:10008C00C48DF084C4FCEF540FC445F0C48DF084CF
:10009C00FFADF0E4CC4FFF22EE8DF08420D2CC7E6D
:1000AC0008CEC5F0CDCBEF2FFFED33FD10D7079B5E
:1000BC005005D5F0F1229BFD0FD5F0EA22C3E49F49
:0D00CC00FFE49EFE22C3E49DFDE49CFC22A7
:00000001FF
